:100000000C9430000C944D000C944D000C944D0059
:100010000C944D000C944D000C944D000C944D002C
:100020000C944D000C944D000C944D000C944D001C
:100030000C944D000C944D000C944D000C944D000C
:100040000C944D000C944D000C944D000C944D00FC
:100050000C944D004C696E6532004C696E65310040
:1000600011241FBECFE5D8E0DEBFCDBF10E0A0E673
:10007000B0E0EAEAF2E002C005900D92A036B107C6
:10008000D9F710E0A0E6B0E001C01D92A036B1079C
:10009000E1F70E944F000C9454010C9400000E9460
:1000A000E5000E94DD0061E081E00E9402018AE536
:1000B00090E00E941C0161E082E00E94020184E560
:1000C00090E00E941C01FFCF0EC000000000000065
:1000D0000000000000000000000000000000000020
:1000E00000000000000001972FEF8F3F920769F793
:1000F0000895CF93DF93EC0104C088EE93E00E9453
:10010000640021978FEFCF3FD807B9F7DF91CF91E8
:100110000895939A81E090E00E946400939881E0B2
:1001200090E00E9464000895992780FF02C0949A8D
:1001300001C0949881FF02C0959A01C0959882FFF2
:1001400002C0969A01C0969883FF02C0979A01C098
:1001500097980E94890008951F93182F82958F7099
:100160000E949400812F8F700E94940082E390E09F
:100170000E9464001F9108951F9310E083E00E9485
:10018000940084E690E00E9479001F5F1330B1F77D
:1001900082E00E94940085E090E00E94790088E26D
:1001A0000E94AC0085E090E00E9479001F910895C4
:1001B00092980E94AC00929A089581E00E94D80023
:1001C00085E090E00E94790008958A9A8B9A92982F
:1001D00093988C9A8D9A8E9A8F9A8FEF90E00E94C6
:1001E00079000E94BC0088E00E94D8000E94DD00D7
:1001F00086E00E94D8008CE00E94D80084E10E9432
:10020000D8000895982F81508230A8F4862F81500D
:10021000803188F4913021F0923029F080E805C0D7
:10022000862F815802C0862F81540E94D80082E315
:1002300090E00E9464000895CF93DF93EC0128C002
:10024000853B61F1863B38F48D3011F1803BB9F08C
:100250008A30B9F41DC0843E51F0853E18F48F3DBC
:1002600081F40BC0863F29F08C3F59F404C081EE25
:1002700016C08FEE14C085EF12C082EE10C08FED55
:100280000EC09927282F882319F0822F0E94AC00D6
:10029000FE0121968491882399F603C084EE282FCD
:0A02A000F4CFDF91CF910895FFCF56
:00000001FF
